:1000000000600020BD020000110300001303000087
:100010001503000017030000190300000000000092
:100020000000000000000000000000001B030000B2
:100030001D030000000000001F030000210300005A
:100040002303000023030000230300002303000018
:10005000230300000000000023030000230300002E
:1000600023030000230300002303000023030000F8
:1000700023030000230300002303000023030000E8
:1000800023030000230300002303000023030000D8
:1000900023030000230300002303000023030000C8
:1000A0002303000023030000000000000000000004
:1000B00023030000230300000000000000000000F4
:1000C0000000000000000000000000000000000030
:1000D0000000000000000000000000000000000020
:1000E0000000000000000000000000000000000010
:1000F0000000000000000000000000000000000000
:1001000000000000000000000000000000000000EF
:1001100000000000000000000000000000000000DF
:1001200000000000000000000000000000000000CF
:1001300000000000000000000000000000000000BF
:1001400000000000000000000000000000000000AF
:10015000000000000000000000000000000000009F
:10016000000000000000000000000000000000008F
:10017000000000000000000000000000000000007F
:10018000000000000000000000000000000000006F
:10019000000000000000000000000000000000005F
:1001A000000000000000000000000000000000004F
:1001B000000000000000000000000000000000003F
:1001C000000000000000000000000000000000002F
:1001D000000000000000000000000000000000001F
:1001E000000000000000000000000000000000000F
:1001F00000000000000000000000000000000000FF
:1002000010B5054C237833B9044B13B10448AFF350
:1002100000800123237010BD6C000020000000004E
:10022000E807000008B5034B1BB103490348AFF3CF
:10023000008008BD0000000070000020E8070000FA
:10024000A3F5803A704700BF174B002B08BF134B34
:100250009D46FFF7F5FF00218B460F461348144AD1
:10026000121A00F099FA0E4B002B00D098470D4B54
:10027000002B00D098470020002104000D000D48FD
:10028000002802D00C48AFF3008000F061FA200093
:10029000290000F047F800F047FA00BF000008000E
:1002A0000000000000000000006000206C00002042
:1002B0008800002000000000000000000E480068D8
:1002C0000E4909680A280AD1002908D10C48026899
:1002D0006FF070031A404FF040031A43026009495F
:1002E000094A0A4B9B1A03DD043BC858D050FBDC7B
:1002F00000F030F8FFF7A8FF3001001034010010C3
:10030000E40E0040F4070000000000206C00002014
:10031000FEE7FEE7FEE7FEE7FEE7FEE7FEE7FEE7B5
:10032000FEE7FEE74FF080430122C3F80025FEE719
:10033000BFF34F8F0549064BCA6802F4E0621343CE
:10034000CB60BFF34F8F00BFFDE700BF00ED00E0C3
:100350000400FA0538B5AF4B1B68591C04BFAE4BFF
:100360001B78062B05D1AD4BAD4A1B68C3F30423A4
:100370001360A94B1B78062B00F03481A54B1B683A
:100380005A1C04BFA44B1B78062B00F08F800A2B4D
:1003900000F08C80A04B1B78062B00F092809D4BC8
:1003A0001B685D1C04BF9C4B1B78062B53D00A2B8B
:1003B00051D0994B1B78062B5AD0964B1A68541C77
:1003C00000F00981974B1B681146062900F08C80CC
:1003D0000A2900F08D80501C04BF8F4B1A78062A22
:1003E00020D00A2A2CD08B4A8E4B12681B68062A12
:1003F00000F0C8800A2A00F0D3804FF01023D3F811
:100400000022002AC0F24981D3F80432002BC0F246
:100410004481854B1B68DB0700F16581834B844A6F
:100420001A6038BD834B7B4A1B681268824903F00F
:100430004F030B60511C04BF774B1A78062AD0D1AA
:100440004FF08043D3F80024D20744BF6FF001027D
:10045000C3F80024C7E74FF080430022C3F80C2103
:10046000C3F81021C3F838256B4B1B78062BA4D199
:10047000724B1B68C3F30313033B042B9DD8704AD4
:10048000D25C12B16F4A032111606F4AD35C002B1A
:1004900093D06E4A6E4C6F496F4B0520106001255A
:1004A00000203F22256008601A6086E76B4B6C4A8B
:1004B0001B68C3F342331360574B1B78062B7FF442
:1004C0006EAF5E4B1B68C3F30313033B042B3FF675
:1004D00066AF644AD35C002B3FF461AF624AD368D5
:1004E00023F08073D3605AE7033B042B40F28B80E8
:1004F0004FF080525D4BD2F80414C3F82015D2F8A7
:100500000814C3F82415D2F80C14C3F82815D2F82F
:100510001014C3F82C15D2F81414C3F83015D2F8FF
:100520001814C3F83415D2F81C14C3F84015D2F8C7
:100530002014C3F84415D2F82414C3F84815D2F88F
:100540002814C3F84C15D2F82C14C3F85015D2F85F
:100550003014C3F85415D2F83414C3F86015D2F827
:100560003814C3F86415D2F83C14C3F86815D2F8EF
:1005700040142848C3F86C15D2F844140268C3F834
:10058000701528E7033B042B7CD93949214A0B68B5
:100590001268244843F480630B600A2A03680BD175
:1005A000002B3FF42AAF24481A4A01681D4B1268F9
:1005B0001B6841F00F010160062A7FF41EAF033B68
:1005C000042B64D94FF010224FF08043D2F8082258
:1005D000C3F8582511E7194B0F491B680978C3F375
:1005E0000313F2E6154B1B68C3F30313033B042B01
:1005F0003FF6C4AE1F4AD35C002B3FF4BFAE1E4B88
:100600001E4A1A60BAE61E49CB5C002B3FF4E3AEEB
:100610006EE700BF30010010E00F00F0240300106F
:1006200040350140340100100C1200100000002081
:100630000090D00358020010E40E0040E80F00F0D4
:10064000DC070000A0050040DC0700001056004059
:1006500088560040185600401456004044020010CE
:100660003C050040DC070000F0ED00E000C0004069
:100670003C170040DC07000074C007400DF0ADBA25
:10068000C4070000244AD25C002A99D07DE7234A9F
:10069000D35C002B3FF4B1AE94E7214A0123C2F8AA
:1006A0000435D2F80034002BFBD04FF01023152175
:1006B0001B4AC3F80012D2F80034002BFBD04FF0D5
:1006C00010231521164AC3F80412D2F80034002B67
:1006D000FBD000231249C2F80435D1F80034002BB6
:1006E000FBD0FFF725FE0E4B0122C3F80425D3F8FB
:1006F0000024002AFBD00B4B094A00211960D2F8D4
:100700000034002BFBD000230549C2F80435D1F892
:100710000034002BFBD0E4E7CC070000D407000036
:1007200000E001400C12001008B5074B044613B15D
:100730000021AFF30080054B1868836A03B1984726
:10074000204600F031F800BF00000000E407000080
:1007500070B50D4D0D4C641BA4100026A64209D1A6
:100760000B4D0C4C00F022F8641BA4100026A6428E
:1007700005D170BD55F8043B98470136EEE755F8B2
:10078000043B98470136F2E7640000206400002033
:10079000640000206800002002440346934200D118
:1007A000704703F8011BF9E7FEE700BFF8B500BF8B
:1007B000F8BC08BC9E467047F8B500BFF8BC08BC42
:1007C0009E4670470000010101000000000000018A
:1007D0000100000000000000010000000100000016
:0C07E000000000000400002000000000E9
:0807EC0054FAFF7F0100000038
:1007F4000090D00300000000000000000000000092
:1008040000000000000000000000000000000000E4
:1008140000000000000000000000000000000000D4
:1008240000000000000000000000000000000000C4
:1008340000000000000000000000000000000000B4
:1008440000000000000000000000000000000000A4
:0C0854000000000025020000010200006E
:04000003000002BD3A
:00000001FF
